:030000000219FDE5
:03000B000200AA46
:03002B0002019936
:03005B0002034F4E
:0300730002033550
:1000800002030406080C10182030406080040608A3
:100090000C10182030406080A0C000070F1F3F0DDB
:1000A0000D0403060D0503030202C2AF306308C24C
:1000B00063857C8AD2AF32C0D0C0E0206227E525BC
:1000C0006002E473E525F4C3334009758A00D26306
:1000D000F57C01D6F58A758B00758D00D262D0E073
:1000E000D0D0D2AF32C3E526334009758A00D2633F
:1000F000F57C01F6F58AC262E526F4603B306803C0
:10010000207213758B00758D00D0E0D0D0C292C2E2
:1001100096C294D2AF32C292C296C294206E0C2084
:100120006609740ED5E0FDE57E4290758B00758DF5
:1001300000D0E0D0D0D2AF32758A00D263757C0097
:10014000C28DD262212B01C4306805206602D29292
:1001500001C4306805206602D29401C430680520CD
:100160006602D29601C4C29330680A2066077410F2
:10017000D5E0FDD29201C4C29530680A20660774AA
:1001800010D5E0FDD29401C4C29730680A206607FA
:100190007410D5E0FDD29601C4C2AFC2AD53E6EFF4
:1001A000C0D0C0E0D2D3D2AFE57D6009E57A60056A
:1001B000757A00413E757A01C2CEE52A6007207447
:1001C00049152A410A7800790020742EE580307E96
:1001D00001F430E50278FF53DACF207E0343DA20C2
:1001E000307E0343DA10C2D8C271E580307E01F45C
:1001F00030E50279FFC3E89970CB306103752A407E
:10020000207403752A40885FD27020740DE52B603E
:1002100004152B411A43DA01C2D8207002412DA8DF
:100220005F206102C270207402412B88227882B65E
:100230000403852224C3E52594404002D26420CFE4
:100240000AD0E0D0D043E610D2AD32C2CF053AE5B5
:100250007D6009E57B6005757B00612B757B01780E
:1002600002E52A6005307402152AC3E55F94014057
:10027000057562004187756300756C00E5622401B5
:10028000F56250037562FF7982B7020D306D1DC3B0
:10029000E52294324016854D227982B7030E306DE7
:1002A0000BC3E52294324004798E8722C3E523955F
:1002B0002260084004152341BB0523D8CA056CE51C
:1002C0006C7002156CD56D63756D017805C3E56CB6
:1002D000956E4057C3E56C956F50087801756D03B6
:1002E0000202EFC3E56C957050057801756D01C38E
:1002F000E5659524401E7982B704026120206D14C3
:10030000852465E56C046003856E6C756D0175234D
:100310003C02032BE5652850057565FF6120F565F6
:10032000E5650470067563FF756CFFD0E0D0D043BF
:10033000E610D2AD32C2AFC0D053E67FC260759135
:1003400000855694855795759104D0D0D2AF32C2AE
:10035000AF53E6EFC2ADC0D0C0E0C0F0D2D3D2AF51
:10036000A8FBA9FCE57D6007C3E913F9E813F8C20F
:10037000D830710261C153DACF207E0343DA1030E6
:100380007E0343DA20D271E580307E01F420E5025D
:10039000619888278928A1A053DACF207E0343DA09
:1003A00020307E0343DA10C2D8C271307402A18CAF
:1003B0007800E580307E01F430E502A18C885FA1F1
:1003C0007453DACF207E0343DA20307E0343DA1001
:1003D000C271206102819A53DACF207E0343DA1082
:1003E000307E0343DA20C2D8D271885A895BC3E8D1
:1003F0009558F8E99559F97B007E087A00C3E8948E
:100400008CE994005005755E00818C882178A2E605
:10041000A8216055C3E894C8E994005008E4D2E4E8
:10042000FB7A0A8167C3E89468E994015008E4D232
:10043000E3FB7A0F8167C3E894D0E994025008E4A3
:10044000D2E2FB7A1E8167C3E894A0E994055008C4
:10045000E4D2E1FB7A3C8167C3E89498E9940850C0
:1004600008E4D2E0FB7A787E00C3E8955CFCE9956D
:0F0470005DFD30E70AECF42401FCEDF43400FDEF
:10047F00755E00C3EC9AED9E5003755E01885C8932
:10048F005D855A58855B597802A174C3E89527F8A2
:10049F00E99528F9307C02A158307B02A158307AB7
:1004AF0002A15120750281BDE9FDE8FC81DCE9C3A1
:1004BF0013F9E813F8307902A151E9C313F9E813DE
:1004CF00F8307802A151E9C313FDE813FC2061262F
:1004DF00C3EC941CED9402400281F3ED7018C3EC51
:1004EF0094C850120529C3E529940A5002A18C75AE
:1004FF005F00D270A18CE529600215297400207F5E
:10050F00037896E624FAFEE43400FFC3EC9EFCED7C
:10051F009FFD500678007900A158C3EC94FFED942D
:10052F0000400678FF7900A158EC8575F0A4C5F05E
:10053F00A2F733F87900400302057478FF790002BF
:10054F000574E9C313F9E813F8307C0EE9600278FB
:10055F00FFC3E81338F8E43400F9C3E894FFE994D3
:10056F0000400278FF885FD270206102A18C741F57
:10057F00F4552F4BF52FC274EB7002D274752A40CD
:10058F00307403752A0A306102A1A020740353DA74
:10059F00FE207403752B20D0F0D0E0D0D0D2AD4325
:1005AF00E6103279010205D079030205D0790A02EB
:1005BF0005D0791E0205D079640205D079C80205ED
:1005CF00D07817E4D5E0FDD8FAD9F6227A147B78E3
:1005DF000205F77A107B8C0205F77A0D7BB40205C2
:1005EF00F77A0B7BC80205F77902B27DE4C295D585
:1005FF00E0FDD294D5E0FDC294D5E0FDD295D5E0D3
:10060F00FDD292E576D5E0FDC2927496D5E0FDD984
:10061F00D9EAF8D5E0FDD8FBDBCEC29522C37C002A
:10062F007D0075F00005F0EA33FAEB33FB50F6EB83
:10063F0013FBEA13FAC3E9FFE8FEE89AF8E99BF91E
:10064F005004EFF9EEF8B3EC33FCED33FDD5F0DFEA
:10065F00EDF9ECF822E889F08A20D2D4F8A9F07BE2
:10066F000030F70B7BFFF42401F8E9F43400F9E8CC
:10067F008520F0A4ADF0F8E98520F0A4AFF0FEEDF1
:10068F002EF974003FFA7C04C3EA13FAE913F9E870
:10069F0013F8DCF48BF030F70AE8F42401F8E9F4EE
:1006AF003400F9E889F0C2D4F8A9F0227882B604B0
:1006BF000302075AC3E55F9419401EE52D540670D7
:1006CF0018206D3678057994E7146007780A14605E
:1006DF00027812C3E54198401F306D098567657533
:1006EF006CFF756D01852224E4F545F546F547F558
:1006FF0048F549C26D02075AD26D7994E714701309
:10070F00E523F43333F913F8E9540104F9E854FEFF
:10071F0002074EE714147014E523F4333333F9133F
:10072F00F8E9540304F9E854FC020756E523F433BF
:10073F00333333F913F8E954070404F9E854F8C3D1
:10074F009440F8E99400F98845894622C3E541139E
:10075F00F9E54013F8C3E54598F8E54699F9500CCB
:10076F00C3E89480E994FF4016020792C3E8947F90
:10077F00E994005003020792787F7900020792787C
:10078F008079FF884A894B22E54A2547F8E54B35A2
:10079F0048F9854B20E4300701F43549FA30E70971
:1007AF00C3EA94F040150207D0C3EA940F50030236
:1007BF0007D078FF79FF7A0F0207D0780079007A97
:1007CF00F0C3E5249564500AC374019524500B02BD
:1007DF0007EEE54B20E70E0207EEE54B30E7068804
:1007EF004789488A492278A4E6FAC3E54A33F8E5EF
:1007FF004B33F9120664E930E70BC3E89480E994B0
:10080F00FF40130129C3E8947FE9940050020129A6
:10081F00787F79000129788079FFE820E715C3E513
:10082F002398F84009C3E894014003020850780167
:10083F00020850E8F424012523F8400302085078F9
:10084F00FF884C2278A5E6FAA848A949120664E960
:10085F0030E70CC3E89401E994FF4016020885C302
:0F086F00E894FFE99400500302088578FF7900B0
:10087E00020885780179FFE920E715C3E54C98F861
:10088E004009C3E8940140030208AC78010208ACA9
:10089E00E8F42401254CF840030208AC78FF8824C4
:1008AE002278FFC26420693D206A12D264C3E541FA
:1008BE00940A4009C3E52594405002C26479A1E729
:1008CE006023E541601F74FF8541F0848539F03067
:1008DE006A0375F005A4F8C5F0600278FFC3E895C9
:1008EE00675002A867886622C3E54094C8E5419424
:1008FE0000E5665003142107046002F56622788332
:10090E00E6F520120FC575E8901205B275E890E570
:10091E00E820ECFBA8BDA9BE12105F7571007572C0
:10092E0000C3740013FD7400606613FC74002CFC8D
:10093E0074003DFDECFAEDFBC3E89AE99B4014E52B
:10094E00712400F571E5723400F572EA2CFAEB3D74
:10095E00FB80E5AE71AF72C3E57213F9E57113F862
:10096E00C3E913F9E813F87A03C3E913F9E813F8A6
:10097E00DAF7AA201A700975710075720002099EC5
:10098E001AEA6008EE28FEEF39FFDAF88E718F72E0
:10099E002275E890227883E6FFE5E820ECF7A8BD03
:1009AE00A9BE0573C3E57394084052757300E9FA46
:1009BE0079A0E76044EA7007E574601B0209D9C3A9
:1009CE00E895746010E5745006600C140209E50495
:1009DE0060F90209E5E574F574C39472401B756401
:1009EE00C0C394044013756480C39404400B7564B3
:1009FE0040C39404400375640075BB0822EFC39492
:100A0E0001601F7400601BC3E894FFE99403501249
:100A1E00C3E89571E995725009E564600C1564029E
:100A2E000A37E564F460020564A864C3E5249850AF
:100A3E0002A824C3E89565400AA865E565F460033D
:100A4E0085656488258826E573B4070375BB102277
:100A5E00743279A687F0A4C5F0A2F733F8C3E895EF
:100A6E00644002A864882288248825882688672204
:100A7E007540007541F022C2AF75C820A8CCA9CD33
:100A8E00AA3A30CF010A75C824D2AFC3EA13FAE9E5
:100A9E0013F9E813F8AB3BAC3C883B893CC3E89BAD
:100AAE00F8E99C20690A547FF930670261A8610554
:100ABE00AD3D8A3DF9EA9D547FFA600478FF79FFD7
:100ACE00AE3EAF3F8B3E8C3FC3EC9FFCC3E99CF523
:100ADE0042A83BA93CC3E89EF8E99FF9C3E5411340
:100AEE00FBE54013FAE82AF540E93BF5415006755F
:100AFE0040FF7541FF614FAA40AB41AC40AD417E16
:100B0E00047F02C3EB940440021E1FC3EB94084003
:100B1E00021E1FC3ED13FDEC13FCDEF7C3EA9CFAB5
:100B2E00EB9DFBEF6009C3E913F9E813F8DFF7EA71
:100B3E0028FAEB39FB8A408B4150067BFF8B408BAA
:100B4E0041C3EB94025002D2673069047F03617A8D
:100B5E007892E6FFC3E537948240110FC3E53794D0
:100B6E00A040010FC3EF940640027F057E03E541CE
:100B7E00C4540FF9E541C454F0F8E540C4540F28AD
:100B8E00F8C3E89EFAE99400FB4009C3EA9402EB2D
:100B9E00940050047A02E4FB61F4AA40AB41EBC42A
:100BAE00FEEAC4540F4EFCC3EA9CFAEB9400FBC35E
:100BBE00E813C313F8EA28FAEB3400FB8A408B41A2
:100BCE00C3EB94024002C2677803EBC4FE7B00EADB
:100BDE00C4540F4EFAC3EA98FA4005C39402500269
:100BEE007A027892E6FF30600261F48552568553A0
:100BFE0057D26043E680C3E49AF8E49BF9C3E83326
:100C0E00F8E933F93067028195E8FAE9FBD3E91385
:100C1E00FDE813FC88528953C3EF94036038EF202C
:100C2E00E00DE82CF8E93DF9ECFAEDFB020C50E88A
:100C3E0028F8E939F9C3E82402F8E93400F97AFE14
:100C4E007BFFC3EF9403400E8A548B55884E894F19
:100C5E008C508D5181C9885489558A4E8B4F8C503A
:0E0C6E008D51306920C3E53394034019E542EF
:100C7C00A2E713F8E555F4240138400B20E708757A
:100C8C0054FFF42401F55581C9E8FAD3E813FC8824
:100C9C0052C3EF94036020EF20E007E82CF8ECFA45
:100CAC0081B5E8282402F87AFEC3EF940340088A41
:100CBC0054884E8C5081C988548A4E8C50E56BC335
:100CCC00335002646BF56B30600281D3753404D2FF
:100CDC006043E680E52D5406601FA840A941C2AFD1
:100CEC0053E67F759100C3E498F594E499F59575F6
:100CFC009104D26043E680D2AF22D2657544007570
:100D0C002000306B03752040020D25D26575440020
:100D1C00752040306B03752000D2AF78012067221C
:100D2C00E52D54066002C265C3E541940540137875
:100D3C000294054008780394054002780630690255
:100D4C00780A206019E544601530690AC3E53394CC
:100D5C00034003D53406D2AFD26CC10891DBD2AFBD
:100D6C000000C2AF20672AE541C3FB940F40027B11
:100D7C000FEB240530730123306A027428206201C2
:100D8C0023F93069027982E58D13E58B13C3994001
:100D9C00B10544E59BF45440B52002A1F230690A38
:100DAC0008C3E8940A400108A14E206502A125C29F
:100DBC006553E67F7591003067107594007595FC4E
:100DCC00759104D26043E680A125AE40AF41C3EEDD
:100DDC0033FEEF33FF50047EFF7FFFC3E49EF59498
:100DEC00E49FF595A1CCC3E53394025002A12530C4
:100DFC006502A125D802C106A14EC26C53E67F75CF
:100E0C009100855494855595759104854E56854F62
:100E1C0057D26043E680D2AFE52D54066008206AB5
:100E2C00020533020E42306C0D206B0A206507154B
:100E3C008115810216BC2278003064053065027879
:100E4C0001E53775F007A4F9E5F028F5F0E9A2F013
:100E5C0013A2F113A2F213F537C39478500375372C
:100E6C0078C3E53795384008D266C292C296C294D0
:100E7C00306002C17C855056855157D26043E68064
:100E8C0022207D11C2AF754302C295D293D2AF75A9
:100E9C009F4002105CC2AF754302C295D297D2AF8D
:100EAC00759F4002105C307243207D20C2AF7543A9
:100EBC0003900177757E20C296C297306204D2945B
:100ECC00C1D0D295D2AF759F4102105CC2AF7543B1
:100EDC0003900177757E20C292C293306204D29443
:100EEC00C1F0D295D2AF759F4302105C207D17C222
:100EFC00AF754303900152C296306202D294D2AFC6
:100F0C00759F4102105CC2AF754303900152C292AF
:100F1C00306202D294D2AF759F4302105C207D11D7
:100F2C00C2AF754304C293D297D2AF759F430210E0
:100F3C005CC2AF754304C297D293D2AF759F410286
:100F4C00105C307243207D20C2AF75430590016662
:100F5C00757E08C294C295306204D292E16CD29331
:100F6C00D2AF759F4002105CC2AF754305900188EB
:100F7C00757E80C294C295306204D296E18CD29771
:100F8C00D2AF759F4002105C207D17C2AF75430530
:100F9C00900148C294306202D292D2AF759F400247
:100FAC00105CC2AF75430590015CC2943062EBD209
:100FBC0096D2AF759F4002105C207D11C2AF754375
:100FCC0006C297D295D2AF759F4102105CC2AF7525
:100FDC004306C293D295D2AF759F4302105C307218
:100FEC0042207D20C2AF754301900188757E80C27E
:100FFC0092C293306204D2960108D297D2AF759FF9
:10100C004302105CC2AF754301900166757E08C245
:10101C0096C297306204D2920128D293D2AF759FB8
:10102C0041015C207D16C2AF75430190015CC292F8
:10103C00306202D296D2AF759F43015CC2AF75434A
:10104C0001900148C296306202D292D2AF759F4194
:10105C00C26622900146757E00C292C296C294C2AC
:0F106C0093C297C295C2622278807607087607F2
:10107B000876010876040876FF0876FF08760A08DA
:10108B007602087601087601788C760108760008DE
:10109B0076B40876FF0876FF0876FF0876030876A5
:1010AB00FF0876010876FF0876250876D008767853
:1010BB000876C80876040876FF08760108760008DB
:1010CB00767A08760A0876010876010876000876A3
:1010DB00FF227887E6FFC272BF0302D2727888C202
:1010EB007DE630E102D27DC27E7889E630E102D224
:1010FB007EC3EF94026008758E01D27302110F75D7
:10110B008E00C273227880E6149000809378A4F648
:10111B007881E6149000809378A5F67886E6149093
:10112B00008D9378A6F6789FE6F8700108C3E894D3
:10113B001140027811E82828F56E256E256E28F5EA
:10114B006F256E2828F570789CE67538FF75390C7D
:10115B00B402067538A075390AB403067538827562
:10116B00390578A3E61490009A93F569115F222252
:10117B007896E6FA7897E6FB7888E6B40305C3EB36
:10118B00940EFB307F047A007BFFC3EB9AFCC39475
:10119B008250027C827575000575EC8575F0A4C3D1
:1011AB00E5F0947D40F222D27F317B1205C17A00AB
:1011BB007B007C101205B7E55F2AFA74003BFBDC61
:1011CB00F37C04C3EB13FBEA13FADCF7FEC27F31AB
:1011DB007B22E5EF20E6037520000520903FFFE51D
:1011EB0020146006901FFF1460009304600375EFDA
:1011FB001253D9BF7581C043FF801205B275EF0240
:10120B0043B203E5B3240420E70DF521E5E320E029
:10121B00068521B343E301115F7580FF75A400754B
:10122B00F13075D4DF75900375A5FC75F2FC75D59F
:10123B000175A60175E241C292C296C2941205C60F
:10124B00D293D297D2951205B2C293C297C295E4AC
:10125B00F8F6D8FD756B01117412170B789886761A
:10126B00753001C2AF1205CB1205DB1205C1120599
:10127B00E21205C11205E91205C112182D1205CB98
:10128B001205CB1205C6C2AF78FA79FA308507D9A9
:10129B00FBD8F7021C0011DD3110317A317B7898C5
:1012AB008676115F75B68075A900757D00758850BF
:1012BB0075891275C82475910475D84075A8227567
:1012CB00B80275E690759B80759D0075D10E75BC47
:1012DB005875BB0875BA1175E8801205B2D2AF12FA
:1012EB00090C53DACF207E0343DA20307E0343DA36
:1012FB001043DA01C2D8C2711205CBD2617B037ADB
:10130B000CE55E70077A0CDB030212911205C1200B
:10131B007003021291C270E55FC3940240E1E52FA6
:10132B00541F856160F561B560D5DAD5C26153DABA
:10133B00CF207E0343DA20307E0343DA10C2D8C2BB
:10134B007178A2E67008D274E52F54E0F52FC275C0
:10135B007529001205C6307409C3E529940A4002A9
:10136B00D2751205B778023074027800C3E55F9826
:10137B0040F0C2AF1205DB1205DB1205DBD2AF1258
:10138B0005CB754D001205B7788CE6C3940150035D
:10139B00021466E530C394015003021466207435C1
:1013AB00C3E55F94FF5003021466C2AF1205F0D27F
:1013BB00AF1205C6C3E55F940150EFC2AF1205DB58
:1013CB001205BC1205DBD2AF1205C6C3E55F94FF55
:1013DB0040E90218B27F05D27F317B1205C6C2AF3E
:1013EB00C27F317BAE5FC3E55F947FD2AF40761295
:1013FB0005B2C2AF1205F0D2AFDFDC31B2C3EE944F
:10140B00057897F61205CB12174C1218357F0AD2B6
:10141B007F317B1205C6C2AFC27F317BAE5FC3E5A6
:10142B005F947FD2AF50E61205B2C2AF1205DB124A
:10143B0005BC1205DBD2AFDFD631B2EE24057896B0
:10144B00F61205CB12174C1218641205C6317BC36A
:10145B00E55F94FF500261A80218B2C3E55F954D9A
:0D146B004003855F4D1205C678017988E7C2
:10147800B403027805C3E55F9840026190C2AF12D9
:1014880005F01205F01205F0D2AF1205CB75300049
:10149800E4F531F5320531E531F470390532789AE1
:1014A800E67819146012783214600D787D1460089B
:1014B80078FA146003753200C3E532984017153284
:1014C8007531B478998676C2AF1205F0D2AF7898A4
:1014D80086761205C61205BCE52A700530740241ED
:1014E8009178012074027806C3E55F9840A7120539
:1014F800C6E52A7003021291C2AF115FE4F522F526
:1015080023F524F525F526F56AD2AF7885E6C333A9
:10151800F568E4F545F546F547F548F549F573F5F9
:101528002CF52DF53775730875BB101205B2120925
:101538009FE5E820ECFBA8BDA9BEE97001F8887416
:101548001209A375730875BB107887E6FE76021139
:10155800DD7887EEF6C2AF7564FF120A5E852264F5
:10156800852265852266D2AF75220175240175250D
:101578000175260185636C756D0175B69075A903B3
:10158800757D017888E6B40307C27D307602D27D86
:10159800D268D269753300120FC5120FEA120A7E9B
:1015A800120A85120A7E120A85120A7E0215C3C221
:1015B800AF11DDD2AF75730075BB08120D17120697
:1015C800BB120E43120E8D120A85120D06306D03E2
:1015D80012075B2067031208AF3067031208F61280
:1015E8000E43120EB2120A85120D17306D03120740
:1015F80097120E43120F29120A85120D06306D0339
:101608001207F5120E43120F4E120A85120D1730EB
:101618006D03120853120E43120FC5120A851209E0
:101628009F120D06120E43120FEA1209A3120A8521
:1016380030692F206B2C85676485676585636C75B9
:101648006D0179187A0CC3E533994009C269D26AE9
:101658008A3502166AC3E55F940140030215C30286
:1016680016C4306A1B206B18E535147004C26AA1D1
:10167800B7F535C3E55F940140030215C30216C4EC
:10168800753600C3E5629401400985676585636C1A
:10169800756D01C3E56278FA985021307404E52A23
:1016A800601A78F0306B058567647820C3E5419847
:1016B8005002A1C30536E55F6002C1C7753600C296
:1016C800AF115F7887E6FE760211DD7887EEF6E4E3
:1016D800F522F523F524F525F526F568C26875B6D3
:1016E8008075A900757D00D2AF1205B2115F307404
:1016F80006E52A70024191788DE6C39401400261A3
:101708006D8198901A0D782012178EE520B4A50CDB
:10171800A312178EE520B45A0302172C117412175E
:101728004C02174B901A0378807B0A12178EA30875
:10173800DBF9901A0F788C7B1812178EA308DBF947
:10174800901A2722C2AF1217CD1217A7901A007449
:101758000E121793A37404121793A37414121793F9
:10176800901A0378807B0A121792A308DBF9901A63
:101778000F788C7B18121792A308DBF91217E01266
:1017880017BE901A2722E493F622E6438F01538F5F
:10179800FD75EF0275B7A575B7F1F0538FFE2243BB
:1017A8008F02438F0175EF0275B7A575B7F1901ACF
:1017B8000DF0538FFC22901A0D74A5F193901A0E18
:1017C800745AF193227A3079D07820901A40F18EA9
:1017D800E520F709A3DAF7227A3079D0901A40E7A2
:1017E800F19309A3DAF922AB77A878BB01027980D3
:1017F800BB02027981BB03027982BB04027994BBE4
:1018080005027983BB06027986BB07027992BB0879
:10181800027987BB0902799CBB0A027988BB0B0253
:101828007989E8F7227C051205CBDCFB22C2AF12CE
:1018380005DB1205E21205E91205F01205BC1205D6
:10184800DB1205E21205E91205F01205BC1205DBF0
:101858001205E21205E91205F0D2AF22C2AF120555
:0D186800F01205E91205E21205DB1205BCC5
:101875001205F01205E91205E21205DB1205BC128C
:1018850005F01205E91205E21205DBD2AF22AE77AB
:10189500AF78C2AF1205DB1205DB1205DB1205BC02
:1018A500DEF21205F01205BCDFF8D2AF22113511B8
:1018B5002D112D75770175780175790011937C05CA
:1018C500AD5F1205CBC3ED955F70F5C3E55F940180
:1018D500400AC3E55F94FF40340218F01217EF1277
:1018E500174C1135C2AF75EF12112DDCD30579C335
:1018F500E5799403500280C4112D0578E57714909D
:10190500009F93F808C3E57898500280AC112D111B
:101915002D0577C3E577940C5002809A1210741246
:09192500174CC2AF75EF12112D31
:0319FD000211DDF7
:101A00000E041407070104FFFF0A020101A55A0191
:101A100000B4FFFFFF03FF01FF25D078C804FF01DA
:081A200000FF0A010100FFFFB5
:101A400023475F556C74726132304123202020207F
:101A500023424C48454C492346333930232020202B
:101A60002020202020202020202020202020202076
:101C0000C2AFC2D353D9BF7581C043B20343FF8073
:101C1000752438752503B1C975EF0275E24043F1AB
:101C20002053A4DF75D400D2857DFA780379E67C51
:101C300010752200752300901DD67B0675249875BB
:101C400025013085028142208508D8FBD9F9DCF7CF
:101C500081B4308508D8FBD9F9DCF781B4B189E4C7
:101C600093A3C39A6004DDC381B4DBDBB17B600264
:101C7000812B7B08E493FAA3B15CDBF87A30B15C8A
:101C8000752200752300B17BEAFCEBFDC3ED94FEE9
:101C9000400EB17B8A278B28ED30E0048A828B834B
:101CA000B17B7AC270D8C3ED94FE601350CEBD00F4
:101CB00025EC60097520007521FF0200008100A855
:101CC00027A9280809D804D90281D3B17FEA89AAB3
:101CD000F281C50D81A0C3ED94035049EDA2E092BD
:101CE000007AC5C3E5829400E583941C50902000DF
:101CF00010438F02438F0175B7A575B7F1F030001F
:101D00001FA827A9280809438F01538FFDD804D99C
:101D100002A12089AAE275B7A575B7F1F0A3A10DBC
:101D2000538FFC817C7AC1BD030CE493A3FAB140CC
:101D3000DCF8B138817C817EAA22AB23B15CEBFA5E
:101D4000EA6222752608C3E52313F523E52213F57D
:101D50002250066323A0632201D526EAB1C9B1C986
:101D600075260AEAF4200102D285300102C285B14B
:101D7000C9C3134002C201D526EB22B17FEAFB2082
:101D80008502A17F308502A184752608AE24AF2587
:101D9000C3EF13FFEE13FEB1CDB1C9C3EA13308513
:101DA000024480FA30E703632201C3E52313F523DD
:101DB000E52213F52250066323A0632201D526D91C
:101DC000E52265236523F52222AE24AF250E0FDE22
:101DD000FEDFFCD20122424C48656C693437316326
:041DE000F390060175
:00000001FF
